:100000000C9434000C9466031895000018950000B9
:10001000189500000C944F021895000018950000E8
:10002000189500001895000018950000189500001C
:10003000189500000C9424031895000018950000F2
:1000400018950000189500001895000018950000FC
:1000500018950000189500001895000018950000EC
:1000600018950000189500008FEF8DBFC0EEE8EDE9
:100070004E2E84E08EBFD4E0F4E05F2EEEEFF3E08E
:10008000A0E0B1E0A89584B7082E877F84BF88E1FF
:100090009927809360009093600088278D93319713
:1000A000E9F70E9469046624229A2A9A569A579A76
:1000B0005F9855985D9A259A209A5298219853985E
:1000C000549880E08093800082E08093810088E1F2
:1000D00080936D00809169008C7F826080936900BD
:1000E000E89AE09ADA9AB09A8CE00E94B7040E94EB
:1000F0005E0480E080930101809100018F778093FE
:1001000000010E945C04E0E4FCE00E945504289891
:10011000A9E2B0E08C9182FBDEF385E090E00E94E2
:100120003B05789484B7877F84BF8FE1809360001C
:1001300087E0809360008091600088608093600019
:10014000A8950027A9E2B0E08C9185FB0EF401E0B0
:1001500040E0041711F00C94300189E190E00E9416
:100160003B050027A9E2B0E08C9185FB0EF401E08D
:1001700040E0041711F00C943001A9E2B0E08C913A
:1001800085FBDEF7F89400910101003011F00C942A
:10019000060181E0809301010E946304EAE4FCE02F
:1001A0000E9455040E945C04E4E5FCE00E945504B2
:1001B000289AE89880916F00816080936F00809109
:1001C0006800846080936800DA9AB09A80E090E0DA
:1001D000909385008093840080E080930201809159
:1001E00000018F778093000180E090E0A8E0B1E00B
:1001F0008D939C935E9A8AEF90E00E943B055E98F7
:1002000082E08093810078940C94300180E08093A8
:1002100001010E94630408E00E9450040E945C04F3
:10022000E0E4FCE00E945504289880916F008E7FE6
:1002300080936F00809168008B7F80936800E89ABC
:10024000E09A809100018F7780930001A9E2B0E0ED
:100250008C9182FBDEF385E090E00E943B05789470
:10026000A89500910101003011F00C9424020027A0
:10027000A0E0B1E08C9187FB0EF401E041E00417AF
:1002800011F00C942202A4E1B1E00D911D912D9189
:100290003C9148EE53E060E070E00E944A05A8E11E
:1002A000B1E00D931D932D933D93A8E1B1E00D9125
:1002B0001D912D913C9140E058E060E070E00E947B
:1002C000DB04A8E1B1E04D935D936D937D93A8E1CC
:1002D000B1E00D911C914AE050E00E940E04A6E0AE
:1002E000B1E00D931C93A8E1B1E00D911D912D910A
:1002F0003C91A6E0B1E04D915D9157FB1EF46FEF8C
:100300007FEF02C0662777270E94B405A8E1B1E01D
:100310000D931D932D933D93A6E0B1E00D911C919B
:10032000033050E0150780E00CF081E08F93A6E0E9
:10033000B1E00D911C91073050E0150781E014F0F9
:1003400009F080E09F918923882311F40C94BC016B
:10035000A8E1B1E00D911D912D913C9145E050E057
:1003600060E070E00E94AF05A8E1B1E00D931D933D
:100370002D933D930C94EC01A6E0B1E00D911C91FE
:10038000083050E0150780E00CF081E08F93A6E084
:10039000B1E00D911C91093050E0150781E014F097
:1003A00009F080E09F918923882311F40C94EC01DB
:1003B000A8E1B1E00D911D912D913C914AE050E0F2
:1003C00060E070E00E94AF05A8E1B1E00D931D93DD
:1003D0002D933D930C94EC01A8E0B1E00D911D919B
:1003E00017FB1EF42FEF3FEF02C022273327A8E1AF
:1003F000B1E04D915D916D917C910E94B405A8E1B1
:10040000B1E00D931D932D933D93ACE1B1E0E8E194
:10041000F1E00E94CA050E946304ECE1F1E0A0EC67
:10042000B4E01127222705E034E00E9471050E9404
:100430004804EEE5FCE00E945504809100018F77AE
:10044000809300010C944D020027A0E0B1E08C9154
:1004500087FB0EF401E041E0041711F00C944D020B
:10046000A7E2B1E0E8E0F1E00E94CF050E9463045A
:10047000E7E2F1E0A0ECB4E01127222705E034E048
:100480000E9471050E944804EEE5FCE00E945504BC
:10049000809100018F77809300010C94A0000F924F
:1004A0001F922F923F924F925F927F92AF92BF9294
:1004B0000F931F932F933F934F935F936F937F936C
:1004C0008F939F93AF93BF93CF93DF93EF93FF935C
:1004D0008FB78F9380916F008E7F80936F00009114
:1004E0000201003011F00C947D0284E690E0AAE055
:1004F000B1E08D939C930C94B702013011F00C94F1
:10050000890282E390E0AAE0B1E08D939C930C9481
:10051000B702023011F00C94950289E190E0AAE054
:10052000B1E08D939C930C94B702009102010330CB
:1005300081E008F480E08F9300910201043081E0B3
:1005400010F009F080E09F918923882311F40C9426
:10055000B1028AE090E0AAE0B1E08D939C930C9404
:10056000B70285E090E0AAE0B1E08D939C93A3E010
:10057000B1E089B18C93A4E0B1E08C9183FB882732
:1005800080F9082FA3E0B1E08C9184FB882780F9E3
:10059000482F0427A5E0B1E00C930091050101303C
:1005A00011F00C94E302A8E0B1E00D911C91AAE0D7
:1005B000B1E04D915C91040F151FA8E0B1E00D93DF
:1005C0001C930C94F102A8E0B1E00D911C91AAE0FB
:1005D000B1E04D915C91041B150BA8E0B1E00D93C7
:1005E0001C93809103018093040180910001806835
:1005F0008093000180E08093020180E090E090937E
:1006000085008093840080916F00816080936F00EB
:100610008F918FBFFF91EF91DF91CF91BF91AF91FC
:100620009F918F917F916F915F914F913F912F910A
:100630001F910F91BF90AF907F905F904F903F9030
:100640002F901F900F9018950F921F922F923F920C
:100650004F925F927F92AF92BF920F931F932F930F
:100660003F934F935F936F937F938F939F93AF933A
:10067000BF93CF93DF93EF93FF938FB78F93009147
:100680000201053010F00C944A03A2E0B1E08C9115
:100690008F5F8C938F918FBFFF91EF91DF91CF91FF
:1006A000BF91AF919F918F917F916F915F914F918A
:1006B0003F912F911F910F91BF90AF907F905F90CE
:1006C0004F903F902F901F900F9018950F921F9270
:1006D0002F923F924F925F927F92AF92BF920F9371
:1006E0001F932F933F934F935F936F937F938F93BA
:1006F0009F93AF93BF93CF93DF93EF93FF938FB706
:100700008F9380E283B95298219898E1ACE0B1E0F0
:10071000983018F4392F992702C038E098504A9B36
:10072000FECF88941999089487954A99FECF3A95F7
:10073000B1F78D93992361F75298219898E1A0E140
:10074000B1E0983018F4392F992702C038E098505A
:100750004A9BFECF88941999089487954A99FECFB1
:100760003A95B1F78D93992361F7A0E1B1E00D912E
:100770001D912D913C91A4E1B1E00D931D932D931A
:100780003C93A6E1B1E00C9107FB00270EF401E0D9
:1007900041E0041711F00C94DF03A4E1B1E00D91E6
:1007A0001D912D913C9140E050E060E071E00E948D
:1007B000B405A4E1B1E00D931D932D933D93809179
:1007C0000001806880930001EF93FF93E0E6F0E082
:1007D0000E942F05FF91EF91E09A8F918FBFFF91BB
:1007E000EF91DF91CF91BF91AF919F918F917F91C9
:1007F0006F915F914F913F912F911F910F91BF90FA
:10080000AF907F905F904F903F902F901F900F90F0
:100810001895F894FFCF00FC10D0089503D01ED097
:1008200001F8F9CF0024E89457FF02C009D068947A
:1008300000F80BD010F80124089502D009D00895D3
:10084000509540954F5F5F4F0895E89417FF0895C6
:10085000009510950F5F1F4F68940895352F242F32
:10086000E894452B11F468940895512F402F0027E8
:10087000112780E1440F551F001F111F021B130B8E
:10088000416018F4020F131F4E7F8A9599F708955F
:10089000A0ECB4E08D91882311F063D0FBCF0895D4
:1008A00080E25FD00A95E1F708950E946D05802DE2
:1008B00011F057D0FACF089580EC59C081E057D09D
:1008C00005D080E854C080E852D0089583E099278D
:1008D000D2C08AEF90E00E943B053D9A3C9A3B9A39
:1008E0003A9A389A399A419885E090E00E943B05FF
:1008F000409845984498439A429A409AEF93FF93C0
:10090000E4ECF0E00E942F05FF91EF914098B0D009
:10091000409AEF93FF93E4ECF0E00E942F05FF91E3
:10092000EF914098A5D0409AEF93FF93E4ECF0E06C
:100930000E942F05FF91EF9140989AD04298409ADB
:10094000EF93FF93E4ECF0E00E942F05FF91EF910D
:1009500040988ED088E20BD08EE009D086E007D098
:100960000895419A829505D004D082D00895419887
:10097000F9CF859510F4429A01C04298859510F4FC
:10098000439A01C04398859510F4449A01C0449855
:10099000859510F4459A01C04598409AEF93FF93CE
:1009A000E4ECF0E00E942F05FF91EF91409808954C
:1009B00000FC05D0089530D005D001F8F9CF37D02C
:1009C0003FD00895842F952FA62FB72FE894452B5D
:1009D000462B472B11F468940895402F512F622F16
:1009E000732F0027112722273327F0E2440F551FCA
:1009F000661F771F001F111F221F331F081B190BB3
:100A00002A0B3B0B416028F4080F191F2A1F3B1FBC
:100A10004E7FFA9559F708950024E89477FF02C0B5
:100A200006D0689400F809D010F80124089512D077
:100A30004F5F5F4F6F4F7F4F0895E89437FF0895E2
:100A400000951095209530950F5F1F4F2F4F3F4F0A
:100A500068940895409550956095709508953197E4
:100A6000F1F70895689462F80895E89462F808959B
:100A700081E090E000C0EF93FF93EE27E82BE92B95
:100A800031F0E0EDF7E03197F1F70197D1F7FF9101
:100A9000EF9108950F921F922F92C801D901489F9C
:100AA00080014A9F90014B9F202C499F100D211DD2
:100AB000321D5A9F202C589F100D211D321D599F09
:100AC000200D311D689F200D311D699F300D789FCD
:100AD000300D2F901F900F900895C89531960020EB
:100AE00008952E2E3F2E992781918D3209F09395EE
:100AF0008823D1F79A95E22DF32D112361F0091780
:100B000018F011F0101B01C0191B28F021F080E231
:100B10008D931A95E9F780818D3219F48D93319672
:100B200004C0222311F08BE28D93091738F031F0C5
:100B3000091B21F080E38D930A95E9F781918D934C
:100B40008823E1F7332351F0EA2FFB2F31963395B9
:100B50008E9182933A95E1F78EE28C930895040F7B
:100B6000151F261F371F0895041B150B260B370B67
:100B70000895000F111F221F331F0895009510952F
:100B8000209530950F5F1F4F2F4F3F4F08950191D4
:100B900010810EC001911191219130810BC0019102
:100BA000108117FF05C03FEF2FEF04C00081112710
:100BB0002227332737FF03C0E1DF8DE28D93CF93E8
:100BC000DF93CF92DF92EF92AA24BB24CC24DD24C2
:100BD000EE2440E2CAE0DD2755E093E38881890FE7
:100BE00087FD9F7083FD907F891B89935A95A9F794
:100BF000C0DFAA1CBB1CCC1CDD1CEE1C4A9551F7A7
:100C0000E894EFE0FF2782910ED0EB30E0F71EF082
:100C100068948A2D0CD088278D93EF90DF90CF9029
:100C2000DF91CF910895982F829501D0892F8F70F1
:100C3000805D26F0803309F4089568948D930895BB
:100C40004D656173757265200000302E3030303094
:100C50002020000043616C696272617400002020F2
:020C6000000092
:00000001FF
